:02000000932843
:080008004328820750344934FB
:1000100043342D3441344434433420345634323460
:100020002E34303431340D340A34003450344934F1
:1000300043342D344C344F34473420345634313427
:100040002E34303430340D340A34003450344934D2
:1000500043342D345234453441344C3456343134E5
:100060002E34303430340D340A3400348207803476
:10007000403420341034940803193B289401940828
:10008000031D3E2808008C00030E83018F00040826
:100090008D0084010A088E008A018B1860280B19D4
:1000A0007B28562810089500FF3094000E088A001F
:1000B0000D0884000F0E83008C0E0C0E8B100900AF
:1000C00017089200920B62280830910018089200DD
:1000D000920B6828061C031006180314900C910B51
:1000E000662819089200920B732819089200920B47
:1000F00077288B1052284F3081000B110130A70256
:10010000031CA802031CA902031CAA0203185628F8
:100110003A08A7003B08A8003C08A9003D08AA002F
:10012000E13096005628831618308100831285012D
:100130000730860083161F308500F1308600831259
:100140004F309700AA30980055309900AA309A0095
:10015000AA309B00AA309C00940196017623762356
:10016000762390308B00A701A801A901AA01AB0159
:10017000482241303602031DC52844303702031D92
:10018000C528B81FC5280130AB008A012B0882079B
:10019000CD284029F928AB01C5288B128B1ACD2810
:1001A0003B203F3015020319E42A15089D00572310
:1001B000613015020319122A673015020319352A16
:1001C000643015020319F5297230150203196C2ADF
:1001D000773015020319B62A693015020319C029B0
:1001E0006F3015020319C929733015020319D1297B
:1001F000C5288B138B1BF92830308B008B17940884
:10020000031913293B203F3015020319E92A150869
:100210009D0057238B128B1A0A2974301502031D77
:10022000C528AB01C52896080319C528B91F1E2982
:10023000003088007C2109089D005723391F26299A
:10024000083088007C2109089D005723B91E2E29FB
:10025000103088007C2109089D005723391E36295B
:10026000183088007C2109089D0057237721C52874
:10027000C13088007C2109089D0057237721C528BB
:100280008B138B1B402930308B008B17940803197C
:100290005A293B203F3015020319E62A15089D0014
:1002A00057238B128B1A512974301502031DC52850
:1002B000AB01C52896080319C528B91F6329013069
:1002C00088007C218D21391F6929093088007C2113
:1002D0008D21B91E6F29113088007C218D21391E96
:1002E0007529193088007C218D217721C528960138
:1002F0009608031D772908003908831688008312A1
:100300003908B400B40EC030B4053414340888047D
:100310007623081508198A29080048224130360238
:10032000031DBD2944303702031DBD29B81FBD2957
:100330004208A4004308A3000908A000A622013037
:10034000C2070318C30741084302031CB12942082E
:1003500040020318B129381BBE293E08C2003F08DD
:10036000C300A3010C30A4004208A000A622A301F0
:100370000D30A4004308A000A6220800AB0108002D
:100380008316F13086008312000006089D00572373
:10039000C5283B208316013086008312150886008D
:1003A000C52806309E00E621031DC52853309D0058
:1003B00057232D0897002E0898002F089900300821
:1003C0009A0031089B0032089C00C5282D3084001B
:1003D000B3013B201508B30715088000840A9E0B63
:1003E000E9293B201508B307080005309E00E621E7
:1003F000031DC52844309D0057232D08B9002E0841
:10040000BA002F08BB003008BC003108BD003A0814
:10041000A7003B08A8003C08A9003D08AA0002303C
:10042000AB00C52803309E00E621031DC5284130DE
:100430009D00572383162D0888008312FC30AD05DC
:100440002D142D0888002E08A6002F08A50089016C
:1004500009089D000815572308192C2A0130A60207
:10046000031CA5020318282AC5283B20831615085B
:1004700088008312FC309505151415088800412268
:10048000C52808150819422A09089D0057230800A5
:10049000A301A401A5010D30A60036308400FE2280
:1004A000A030A2000E232308A2000E232408A200DD
:1004B0000E23FE22A130A2000E232D23200880004F
:1004C000840A0130A6020130031CA502031C692A1C
:1004D0005D2A34230723080004309E00E621031D13
:1004E000C5282D08A4002E08A3002F08A600300858
:1004F000A50052309D0057230130A602031CA5021F
:10050000FE22A030A2000E232308A2000E232408FE
:10051000A2000E23FE22A130A2000E232D232008CC
:100520009D0057233B2015082002031DA42A0130FB
:10053000A602031CA50203188E2A342307232008D1
:100540009D0057233B20C5280723C528F622FE22FD
:10055000A030A2000E232308A2000E232408A2002C
:100560000E232008A2000E230723080004309E005B
:10057000E621031DC5282D08A4002E08A3002F087E
:10058000A6003008A50057309D005723FE22A0305A
:10059000A2000E232308A2000E232408A2000E238B
:1005A0003B201508A2000E230723F62215089D0004
:1005B00057230130A4070318A3070130A602031C28
:1005C000A5020318C62AC528AC01EB2A1030AC00DE
:1005D000EB2A2030AC008A011030B3002C08052033
:1005E0009D005723AC0AB30BEE2AC528FE22A0308B
:1005F000A2000E2307232218F62A0800861552238C
:10060000061552238611522306115223080006159F
:100610005223861552230611522308000830A100E8
:10062000A20D031C861103188615522306155223AA
:100630000611A10B102B8316F9308600831252236A
:1006400006157623A2018619A2038316F1308600CF
:10065000831206115223861108003B2386110615CA
:1006600052230611522308003B23861506155223F8
:100670000611522308000830A1008316F9308600C5
:10068000831206155223861D031086190314A00D2C
:1006900006115223A10B412B8316F13086008312E1
:1006A00052230800532B542B552B562B08008B1329
:1006B0008B1B572B86101A089F009F0B5D2B083051
:1006C0009E009D0C031C8610031886141B089F00B7
:1006D0009F0B682B9E0B612B6D2B6E2B6F2B861443
:1006E0008B171C089F009F0B732B08001330B4005E
:1006F0005B30B5000000000000000000B50B7A2B55
:06070000B40B782B080089
:02400E00F23F7F
:00000001FF
